:020000040000FA
:20000000A305C305000A4000C707080DE707040D6507020D0607010D8F0000086706120A8E
:20002000C305260AA404C4044000C707080DE707040D6507020D0607010D2F00E706220A58
:200040004507370AE201AD0A270B390A390A390A390A390A390A330A350A390A390A390A70
:20006000390A390A390AA305950AA3052C0AA305000A61001A0C020004006100F00C2100D5
:20008000000000000000000000000000000000000000000000000000000000000000000060
:2000A000000000000000000000000000000000000000000000000000000000000000000040
:2000C000000000000000000000000000000000000000000000000000000000000000000020
:2000E000000000000000000000000000000000000000000000000000000000000000000000
:081000000000000003000500E0
:021FFE00F20FE0
:00000001FF
